:020000040000fa
:080000000414040000000000dc
:020000040000fa
:1004000000000000000000000000000000000000ec
:1004100000000000000000000000000000000000dc
:1004200000000000000000000000000000000000cc
:1004300000000000000000000000000000000000bc
:10280000ffffff00ffffff000fc12000807f2400bb
:1028100000018800000000000a0007001100070006
:10282000000020000000e000020032000000020072
:1028300000000000f82d0200000000000040da0057
:102840000000fe004440a900402b20000000e000f2
:102850000300320000002000a00188004440a800ce
:1028600000000600c0e92200010020001600370029
:1028700062004000e0804800910188009001ba00a9
:1028800062004000e0804800910188009002ba0098
:1028900062004000e08048000002eb006028e10098
:1028a00005003a008301e9000700330003800900b6
:1028b0000059eb00040037006128e10001003200fc
:1028c0000082eb0005000700910188001001ba00aa
:1028d0000200e000e6ff3a000000050091018800d8
:1028e0008002780062004000e08048003559ba005c
:1028f0008301e900080032002559ba008301e9008c
:10290000050032000400e000f4ff320015d9ba00df
:102910008301e900f1ff3a0000000600f8270400f7
:1029200000000000e027040000000000d827040099
:1029300000000000ca27040000000000662a04000e
:1029400000000000122d040000000000442c0400d0
:042950000000000083
:020000040000fa
:020000040005f5
:0457f800fe9300001c
:020000040000fa
:020000040005f5
:0457fc007f3e0000ec
:020000040000fa
:102954001201000010010000000000000008000047
:10296400d80400000900000001000000010200007a
:102974000001000009020000200000000101000025
:1029840000c0000032090000040000000002000042
:102994000806000050000000070500008102000046
:1029a4004000000001070000050100000240000093
:1029b40000010000040300000904000034030000c7
:1029c4004d00000069000000630000007200000078
:1029d4006f00000063000000680000006900000050
:1029e400700000002000000054000000650000009a
:1029f40063000000680000006e0000006f0000002b
:102a04006c0000006f000000670000007900000007
:102a140020000000490000006e0000006300000078
:102a24002e0000003a0300004d0000006900000081
:102a340063000000720000006f00000063000000eb
:102a44006800000069000000700000002000000021
:102a54004d000000610000007300000073000000de
:102a64002000000053000000740000006f0000000c
:102a740072000000610000006700000065000000b3
:102a84002000000044000000720000006900000003
:102a94007600000065000000bc940000dc94000097
:102aa400e094000014950000009500000000000070
:102ab4000000000001f90000000000000000000018
:102ac40009af000000000000010000000a1b000024
:102ad40000000000010000000cc300000000000022
:102ae400000000000daf0000020000000000000024
:102af40010ff0000000000000000000011ff0000b3
:102b0400000000000100000012ff000000000000af
:102b14000100000018ff0000000000000100000098
:102b240019ff0000000000000100000020ff000069
:102b3400000000000000000021ff00000000000071
:102b44000000000022ff0000000000000000000060
:102b540023ff0000000000000000000024ff00002c
:102b6400000000000000000025ff0000000000003d
:102b74000000000026df000001000000000000004b
:102b840031890000010000000000000029e5000078
:102b94000000000000000000377300000000000087
:102ba400000000003a2500000300000000000000bf
:102bb4003b25000000000000000000000080000031
:102bc4000402000020000000000000004d69000025
:102bd400637200006f630000687000004d610000c4
:102be4007373000020530000746f000072610000d2
:102bf4006765000020200000202000003030000025
:042c0400303100006b
:020000040000fa
:102c08000200fa00f00f200070248800f00f200066
:102c180050248800f009200080248800b00f20008c
:102c2800602488008804a80000c020004800de0056
:102c3800c02488009424a8009424a9000000eb0074
:102c4800b02488000040eb00004f780007003700f0
:102c58001e80fb00c200dd0000c020000081400093
:102c68006000b8000089be001e4fe80030c0b30005
:102c78009e4f1000f6ff3600d00020005025880037
:102c880003003700a048200031c0b300a7040700a4
:102c98008ac4bf00684060000004e000f9ff3a0001
:102ca8000040eb0014e8b700818120000040eb00f1
:102cb800a040980094a4a90040c0200000418800ca
:102cc8000040eb0011e8b7000040eb0010e8b70047
:102cd8000080fa00000006000200fa0010c8bf00d9
:102ce8000004e00010003a000000eb00a024880077
:102cf8000000eb0060248800010037009404a8005d
:102d080094c4bf00614060000004e000fbff320093
:102d180010c0b30010e8b7000000eb0030258800b1
:102d2800000120004025880010c8bf00e14f500076
:102d380008003a00f00f2000502488000000eb0043
:102d4800602488008c04a8008c84a80020c0b300ec
:102d580010e8b70080c4bf00704060000004e000c5
:102d68000500320082c4bf00704060000004e0002b
:102d7800010032008200070088c4bf006240600082
:102d88000004e0005c003a008ac4bf0061406000b3
:102d98000004e000150032008cc4bf0061406000f0
:102da8000004e0001100320095ff070040c0b300a6
:102db80010e8b700008020001060880080c0b300d1
:102dc80000ecb70011c020009140780030c0b3007b
:102dd80000c0600001ecb70011c0200091407800ed
:102de800c0c8b30000c0700001ecb7008ac4bf00bf
:102df800704060000004e000050032008cc4bf0091
:102e0800704060000004e000010032005400070038
:102e18008ac4bf00644060000004e000080032007b
:102e28008cc4bf00644060000004e000040032006d
:102e38009e0b0700a048200021c0b3003b040700f8
:102e48008ac4bf0001c8b300014060000004e0006c
:102e5800060032008cc4bf0001c8b3000140600006
:102e68000004e00001003200250007008ac4bf000a
:102e7800624060000004e000070032008cc4bf001c
:102e8800624060000004e000030032008a0b070083
:102e9800f00f20007024880010c8bf00e34f5000d6
:102ea800150036008cc4bf00684060000004e000d4
:102eb800110032000040eb00004f78000b00370093
:102ec8008ac4bf00684060000004e0000a003200c5
:102ed8009024800062eab700a048200031c0b30007
:102ee800120407002e0007001e4fe80030c0b30090
:102ef8009e4f1000f2ff36000080fa000000060026
:102f08000000fa00aac4bf00624060000004e000ac
:102f18000e003200a05280009040900000c8b3001c
:102f280080cf500008003a00004180009040900097
:102f380040c8b30080cf500003003a00a15280007f
:102f4800c0c8b30090409800aa24a900a048200057
:102f580021c0b300f50307000080fa000000060056
:102f68000000fa008284a800a048200041c0b300f5
:102f7800ee030700470b07000080fa000000060078
:102f88000000fa00460b07008284a90000482000d0
:102f980041c0b300e50307000080fa000000060006
:102fa8000000fa0062cabf008080fb00b0ff2f005b
:102fb800008060000000e0001b003a0062cabf0009
:102fc8008080fb00c00f2000008060004280de008f
:102fd8004200dd008000780000c020000080400032
:102fe800a0528800a0528000b052880061a520003d
:102ff80060a520001040780080487800a05280002a
:1030080010409000c2c3b3008240600040c3b300c8
:1030180080cf500002003a000c000700090037007a
:10302800210007000700370062cabf008080fb004c
:10303800b0ff2f0000806000e80f500001003a0048
:10304800220007000080fa00000006000000fa00d5
:10305800004180009040900000c8b30000c06000ac
:103068000004e00003003200014180000040eb0052
:10307800904098000040eb005ceab7000040eb008d
:103088005deab7000000eb00b04088000040eb00ac
:1030980014e8b7009a0007000a0b0700c8010700e8
:1030a8000080fa00000006000000fa005dcabf00b8
:1030b800e24f500002003a00770207000100370093
:1030c800370007000080fa00000006000200fa003e
:1030d80000418000104090000080fb004600de00a8
:1030e80061406000004f78000182200000822000cb
:1030f800104078008048780010c8bf00e84f5000a2
:103108000c003a0000802000204090000080fb0066
:10311800b0248800b02480000000e00003003200e2
:1031280000c1b30010e8b7000200370040c0b30088
:1031380010e8b7005dcabf00e14f500015003a0023
:103148000041800081802000110098000b020700d8
:103158005ccabf00e24f500004003a000141800001
:1031680040c8b300904098000b0037001e04e000f0
:1031780004003a000141800080ccb30090409800e0
:10318800050037000141800080c8b30090409800d6
:1031980001003700020007000080fa000000060066
:1031a8000400fa005dcabf00e24f50002e003a004a
:1031b80094c4bf000042b2000004e0002a003200bc
:1031c800a052800010407800e84f500026003a00d6
:1031d800a052800010409000c2c3b300824060003b
:1031e80040c3b30080cf50001f003a00b0528000a7
:1031f8009040900000c8b30000c060000004e000e8
:1032080019003a00b0528000018020001100980097
:103218000040eb00204798000f0037002e40900038
:103228000080fb00800078000080200000814000c2
:103238002e4090000080fb008000780080802000f5
:103248000080400010407800004978002e4090002f
:103258000040e800204798002e409000e74f5000bb
:10326800eeff3600130037000040eb005deab700c0
:10327800b152800080c0b30080487800b15280000d
:103288000080200090009800b1528000c0c8b300b0
:1032980090409800014180000040eb009040980069
:1032a80000418000000f78009e0078000040eb008d
:1032b8009040980080812000900090000008200035
:1032c800008060000000e0000b00320080812000d8
:1032d800300090000000e0000300320080812000f0
:1032e8003000900000000100818120001100900052
:1032f8000070a100900098000080fa00000006000d
:103308000400fa0000802000104078000046b20057
:103318000004e00043003a000080200010409000c4
:103328000080fb006101b900028fbe00b0002000e0
:10333800010020001e01be00800f5100818f59003e
:1033480038003e001e00be00006001001a00370071
:103358001b003700330037001900370031003700f1
:1033680006003700090037002d0037000b00370032
:1033780008003700140037001f00370014e8a800c1
:1033880080c0b30010e8b700260037008a000700a5
:10339800240037000d0207002200370010812000aa
:1033a800904088001408a80010c0b30016e8b700c1
:1033b80014e8a8001b003700ba00070019003700fe
:1033c8001a000700170037000080200040409000d6
:1033d8000080fb008000780020a5200000804000cd
:1033e800904088001408a80010c0b30016e8b70081
:1033f80014e8a8000b00370014e8a800008020009b
:10340800404090000081fb0000802000a040900018
:1034180020a5200000004100014878000100370085
:103428002c0a07000080fa00000006000600fa00d7
:103438000080200020409000e14f50000f003a002b
:1034480000802000104078007f4060000004e00009
:103458000a003a0014e8a8000080200010409000fc
:10346800e34f500003003a0010002000005388008a
:10347800020037000000eb000053880000802000a5
:10348800204090000004e00049003a00008020003d
:10349800104078007f406000e24f500044003a003e
:1034a80000802000404090006f4060000004e00071
:1034b8003f00320014e8a8000040eb00004f7800fd
:1034c8003800370000c02000200798000080200046
:1034d800404090006f4060000080fb00000040000a
:1034e8008000780000802000404090000080fb00b1
:1034f8004700de000080fb00008040004200dd0045
:10350800800078002e0090000100400020079800fd
:103518000080200010409000e34f500004003a0063
:10352800ae00900040c8b300904098001c003700df
:1035380000802000404090006f4060000080fb0049
:103548000000400080007800a04a20000080400071
:10355800100798001e00900090007800d0ff2f0000
:10356800808060001e009000010878000080200024
:10357800c040900000c8b30000c060000004e00034
:1035880004003200ae00900000c4b30090409800e0
:1035980003003700ae00900080ccb3009040980044
:1035a8001e4fe80010c0b3009e4f1000c5ff360044
:1035b8000080fa00000006000200fa0000802000e7
:1035c8009040780000c8b30080cf500033003a0024
:1035d80000ccb30014e8b700008020003040900011
:1035e8000080fb00000f78001e007800e20f5000fa
:1035f8000c0032001e007800e30f50001700320064
:103608001e007800e10f5000010032002100370051
:10361800a04a29009040880020012000b04088007e
:103628001e00370000802000204090000080fb0032
:103638000000400080007800e0542900008040002d
:103648001000780090408800904080000080e800da
:1036580010007800b040880010003700008020007b
:10366800204090000080fb000000400080007800af
:103678000055290000804000100078009040880024
:1036880090408000104078000080fb00b040880027
:10369800020037000040eb0014e8b7000080fa0091
:1036a800000006000400fa000040eb0008e8b7003c
:1036b8000040eb0009e8b700008020009040780047
:1036c8007fc060000080fb00100798001e0090007b
:1036d800e10f5000120032009e009000e28f50006f
:1036e800110032001e0090000000e00001003200ce
:1036f8002700370014e8a80008c8bf000004a0008d
:1037080008e8b70000538000e10f500020003a009d
:1037180008c8bf000014a00008e8b7001c00370064
:1037280014e8a8001a00370014e8a80000c0200018
:10373800000f780000802000404090006f4060003b
:103748000080fb000000400080007800008020001e
:10375800404090000080fb004700de000080fb0036
:10376800008040004200dd001e0f40001e0078006f
:10377800104090000080fb004200de006100600005
:103788000004e0000200320010c0b30008e8b700ef
:10379800a040800001082000010060000000e00057
:1037a8000500320080802000904088001408a8009e
:1037b80020c0b30016e8b7000080fa000000060039
:1037c8000000fa0094a4a900a0408000010820008d
:1037d800010060000000e00025003a008081200020
:1037e8009000900000082000008060000000e000c9
:1037f8001200320020c0b3005deab700014180002a
:103808000040eb00804878000141800080ccb30084
:1038180090409800b152800080c0b3008048780082
:10382800b15280008080200090009800b152800042
:1038380080ccb300904098004e003700b152800011
:1038480080c0b30080487800b1528000008020001a
:1038580090009800b1528000c0c8b3009040980012
:103868000141800040c8b3009040980041003700f3
:1038780080812000900090000008200000806000f7
:103888000000e0003b003a000080200090407800f3
:1038980000c8b30000c060000004e000240032004b
:1038a80000802000b0009000b0408000808f500061
:1038b800030031000080200030009000b0408800f4
:1038c8002e00070010c0b3005deab700b1528000b7
:1038d80080c0b30080487800b1528000008020008a
:1038e80090009800b152800000c8b3009040980042
:1038f800a152800080c0b30080487800a1528000a7
:103908000080200090009800a152800000c8b300f9
:10391800904098000141800080802000900098002d
:103928000141800080ccb30090409800110037001e
:1039380020c0b3005deab700014180000040eb0001
:10394800804878000141800080ccb3009040980006
:10395800b152800080c0b30080487800b152800026
:103968008080200090009800b152800080ccb30085
:10397800904098000080fa00000006000200fa005b
:10398800b0408000e70f50000e003e00b0408000bd
:10399800000f78005ccabf000004e00003003a0092
:1039a80010c0b3005ceab700080037005ccabf006b
:1039b800e14f500005003a0020c0b3005ceab700b0
:1039c8000200370080002000000f780002418000cc
:1039d80000418000904090001e40900000c07000a0
:1039e80010419800014180001e407800804878000e
:1039f800b14080001e00780000805000b040880070
:103a080080802000f0528800a040800061006000a3
:103a18000000e0001b003a000b003700f152800064
:103a28009240800012407800804878000100e80049
:103a3800f05288000200e800904088001e007800dc
:103a48000000e900000f78001e0078000000e00088
:103a5800f2ff3a000e003700f152800092408000d9
:103a680012407800804878000100e800f052880091
:103a78000200e800904088001e0078000000e9007d
:103a8800000f78001e0078000000e000f2ff3a0006
:103a98000080fa00000006000200fa00a052800030
:103aa80090407800114798001e4090008080fb00ed
:103ab8008081200020009000808f50000400360094
:103ac80080812000200090001047980007003700f0
:103ad80080812000a00090001e4090000080fb0024
:103ae8008080500080812000210098000040eb0079
:103af800004f78000b00370080812000100178000b
:103b08009e80fb00808020000080400010407800ec
:103b1800004978008200e8008081200001087800d0
:103b28001e4fe8001e4090009e4f1000f2ff390023
:103b380080812000200090000000e0001300320087
:103b4800b152800080c0b30080487800b152800034
:103b58008080200090009800a052800010409000c3
:103b68000044b2000004e00004003a00b1528000b2
:103b780080ccb3009040980012003700b15280000a
:103b880080c8b300904098000e003700b152800002
:103b98000080200090009800808120003000900074
:103ba8000000e00003003200808120003000900017
:103bb8000000010081812000110090000070a10028
:103bc800900098000080fa00000006000000fa004b
:103bd80014e8a8000040eb0052eab700008020007b
:103be8002040900011e8b70000802000204090009d
:103bf8000004e00003003a0000c1b30010e8b70079
:103c08000300370000c2b30010e8b700340807000b
:103c18000080fa00000006000400fa00204798001f
:103c28003147980000c02000000f78002e40900017
:103c38000080fb0000004000800078003e409000bb
:103c48000080fb00008040004200dd004200de00f2
:103c58004200dd001e0f40009e00780011409000d9
:103c68000070a100904098003e4090000004e000e1
:103c780007003a002e4090000080fb0080004000c2
:103c880080a52000008040001e087800060037004c
:103c98002e4090000080fb00800040000082200041
:103ca800008040001e0878009e00780011409000b7
:103cb8000060a000904098000080fa000000060014
:103cc8000400fa0020479800314798002e409000e1
:103cd8000080fb000000400080007800a04a20001f
:103ce80000804000000f78003e4090008080fb007c
:103cf8001e007800010878003e4090000080fb001c
:103d08004300de00610060000004e00003003200b0
:103d18008040eb002e409000bfff07003e4090001f
:103d28000080fb004200de00610060000004e0004b
:103d38000300320011c0b3002e409000b6ff070008
:103d48000080fa00000006000400fa0020479800ee
:103d5800314798002e4090000004e0000d003a0022
:103d6800b152800080c0b30080487800b152800012
:103d78000080200090009800b1528000c0c8b300b5
:103d8800904098000141800040c8b30090409800de
:103d9800120037002e4090000080fb000000400019
:103da800800078003e4090000080fb0000804000ca
:103db8004200dd008000780000c020000080400044
:103dc800000f78001e0078009040900040c8b300b3
:103dd80080c070001e007800114098000080fa0032
:103de800000006000800fa002047980031479800b4
:103df80022079800634798003e4090000004e000c6
:103e0800070032002e4090000080fb008000400038
:103e18000082200000804000100f78000600370064
:103e28002e4090000080fb008000400080a520000c
:103e380000804000100f78001e007800904090002d
:103e480000c4b30080c068001e00780011409800cc
:103e58001e007800ae009000110098001e00780047
:103e68006e419000024878001e00780010409000d3
:103e780002c4b300824060001e0078001140980020
:103e88001e0078009040900080c8b30080c0700089
:103e98001e007800114098003e4090000004e000a9
:103ea800100032002e4090000080fb00000040000f
:103eb8008000780000822000008040000001780027
:103ec8002e4090000080fb00000040008000780039
:103ed80000822000008040001040780000497800ef
:103ee8000f0037002e4090000080fb0000004000cb
:103ef8008000780080a52000008040000001780044
:103f08002e4090000080fb000000400080007800f8
:103f180080a520000080400010407800004978000b
:103f28001e0078000080fa00000006000400fa0075
:103f3800000f7800214798002e4090008080fb00f9
:103f4800100020000100dd00804078001e0078008d
:0c3f5800014878000080fa00000006001c
:020000040000fa
:103f64000000fa000000eb00505588004282200057
:103f740003c4b3008040eb0010c0b3009aff0700f5
:103f8400405588000040eb0070eab7006000b800bc
:103f940080558800915588006000b800a0558800bd
:103fa400b15588000000eb00705588000040eb001c
:103fb4007feab70014003700f055800000000100cc
:103fc4000004e0000c003200c05580000000010035
:103fd4000004e000080032007fcabf008080fb00bc
:103fe400100020000100dd00800078007055800082
:103ff4000080700070558800af0307007fcabf00bf
:104004000040e8007feab7007fcabf000004e00078
:10401400e9ff32000080fa00000006000000fa0008
:1040240000802000104078007f406000e14f500085
:1040340013003a0000802000404090000004e0009b
:104044000f003a0000802000104090008080fb00a8
:10405400e00f2000808f500001003200080037007c
:104064000040eb0008e8b700808020009040880002
:1040740010002000b040880010ccb30014e8b70052
:104084000080fa00000006000400fa0070cabf00b5
:104094000080fb00100798001e009000e10f500004
:1040a4006d0032001e009000e10f500004003c003f
:1040b4001e0090000000e000080032009c00370061
:1040c4001e009000e20f5000690032001e009000b4
:1040d400e30f500076003200950037004055800011
:1040e4000000e0000600320040558000904090003f
:1040f40000c8b30000c060000004e0008c003a0077
:10410400204180003141800090538800a1538800f1
:104114004041800051418000b0538800c153880061
:104124006041800071418000d0538800e1538800d1
:1041340030c8bf007eeab70031c8bf007feab700cd
:1041440032c8bf0080eab7000040eb00004f78009f
:104154000a0037001e81fb001e80fb00ee004000b9
:1041640040822000008040009040900000a8200081
:1041740000004100114098001e4fe80032c8bf0003
:104184009e4f5000f3ff3e004055800010407800e1
:1041940092eab70092cabf00ff4f500064003a0091
:1041a40092538000a353800050352500213424000d
:1041b400800f5100818f59005d003a007fcabf0013
:1041c400ef4f50005a003e0080cabf00f04f50002d
:1041d40057003e0080cabf000004e00054003200d3
:1041e4007ecabf000004e00005003200e1a7200001
:1041f4009140780000c8b30080cf50004c003a00d2
:10420400b0538000c153800040428800514288006e
:104214005035250021342500204288003142880091
:10422400e1a720009140780000c8b30080cf50007f
:1042340003003a0010c0b30070eab7003c00370036
:104244007ecabf000004e00039003a0020c0b30079
:1042540070eab70036003700ac010700e14f4000b8
:1042640033003a0030c0b30070eab70030003700c2
:10427400a6010700e14f40002d003a0050c8bf00de
:104284000004e00007003a006042800071428000b0
:10429400e00f5000e08f58000200320020c0b3004d
:1042a40050e8b70030c0b30070eab7002000370010
:1042b400505580000000e000060032005055800098
:1042c4009040900000c8b30000c060000004e0000b
:1042d40017003a0042842000d3c0b30011c0b300d9
:1042e40010c0b300c0fe0700505588004055800040
:1042f4000000e0000600320040558000904090002d
:1043040000c8b30000c060000004e00006003a00ea
:104314004282200003c2b3008040eb0010c0b3000f
:10432400b1fe0700405588000040eb0070eab7007a
:1043340070cabf000080fb000080fa000000060085
:104344000c00fa00cccabf000080fb0050079800a4
:104354005e009000fe0f50009e003200de009000d0
:10436400fe8f500014003c005e009000f20f5000dd
:1043740032003200de009000f28f500007003c0053
:104384005e0090000000e000a9003200de00900012
:10439400e38f500065003200d50037005e009000c6
:1043a400fa0f50007a003200de009000fb8f5000bc
:1043b400b0003200ce003700a0022000de009000e2
:1043c400808f500053003200a0022000de009000d5
:1043d400808f500009003c0050022000de00900055
:1043e400808f50002300320080022000de00900005
:1043f400808f500041003200bd003700d00f2000f4
:10440400de009000808f5000a2003200f00f2000e8
:10441400de009000808f500005003200f002200082
:10442400de009000808f500092003200b000370010
:1044340081cabf00cceab700bd003700005e290086
:104444002185200023000900b05878004002b10003
:104454004002200001002000604288007142880070
:104464000040eb0050e8b700d0cfb300cceab7006f
:10447400af0037000040eb0050e8b700d055800093
:10448400000001003007980041079800e0558000c3
:104494000000010001002000100798002107980087
:1044a4001e48900052e8b7000e48900053e8b70049
:1044b4007e40900054e8b7006e40900055e8b70085
:1044c4005e40900056e8b7004e40900057e8b700b1
:1044d4003e40900058e8b7002e40900059e8b700dd
:1044e40080002000010020006042880071428800a2
:1044f400d0cfb300cceab7008d0037003b010700f2
:104504000004e0008a003a0000c0eb00cceab700e7
:1045140087003700cf0107000004e00084003a0060
:1045240000c0eb00cceab700810037000040eb008c
:10453400004f78000a0037001e81fb009e80fb00bc
:1045440030a92000008040001040780080407800ae
:104554002085200000004100014878001e4fe8003b
:1045640010c1b3009e4f1000f3ff3600200120005d
:104574000100200060428800714288000040eb0086
:1045840050e8b700d0cfb300cceab70068003700da
:1045940020c0b30052e8b7000040eb0053e8b70076
:1045a4000040eb0054e8b7000040eb0055e8b700ca
:1045b4000040eb0050e8b70040002000010020005c
:1045c4006042880071428800d0cfb300cceab700c3
:1045d40057003700f0558000000001000004e0009f
:1045e400060032000040eb0050e8b7006000b8005d
:1045f40060428800714288000a003700950aa900c9
:10460400952aa800954aa900956aa900a0c3b300f9
:104614009feab7000040eb00a0eab70010c0b30067
:1046240050e8b70000c0eb00cceab7004000370008
:1046340095cabf006f406000e64f500006003a0084
:1046440050c8bf00e14f500003003a0000c0eb0027
:10465400cceab70036003700170207006000b80044
:10466400604288007142880000c0eb00cceab700c9
:104674002f0037000040eb0050e8b7006000b8009e
:10468400604288007142880000c0eb00cceab700a9
:1046940027003700505580000000e000060032007b
:1046a400505580009040900000c8b30000c06000e6
:1046b4000004e0001e003a00604280007142800065
:1046c400228520008041780011c0b30010c0b300df
:1046d400c5fd07005055880000c0eb00cceab700c8
:1046e4006000b80060428800714288001000370002
:1046f400f1010700950aa800952aa900954aa80087
:10470400956aa90000c2b3009feab7000040eb001d
:10471400a0eab70010c0b30050e8b7006000b800ca
:104724006042880071428800d0cfb300cceab70061
:104734000080fa00000006000400fa00cccabf00a2
:104744000080fb00100798001e009000f20f50003c
:104754003d0032009e009000f28f500007003c00a4
:104764001e0090000000e000320032009e00900025
:10477400e38f50000d0032005b003700d00f2000a3
:104784009e009000808f500040003200f00f200007
:104794009e009000808f5000390032001e0090006f
:1047a400fe0f5000230032004f003700c201070003
:1047b400950aa900952aa800954aa900956aa90016
:1047c400a0c3b3009feab7000040eb00a0eab70023
:1047d4000040eb00004f78000a0037001e81fb0008
:1047e4009e80fb0030a9200000804000104078002b
:1047f40080407800208520000000410001487800b6
:104804001e4fe80011c1b3009ecf1000f3ff360025
:1048140020012000010020006042880071428800cd
:104824000040eb0050e8b700d0cfb300cceab700ab
:104834003400370010c0b30050e8b70000c0eb00ec
:10484400cceab7002f003700005e29002185200044
:1048540023000900b05878004002b1004002200053
:104864000100200060428800714288000040eb0093
:1048740050e8b700d0cfb300cceab700210037002e
:1048840081cabf00cceab7001e0037005055800033
:104894000000e00006003200505580009040900077
:1048a40000c8b30000c060000004e00015003a0036
:1048b400604280007142800022852000804178009f
:1048c40011c0b30010c0b30047fd07005055880065
:1048d40000c0eb00cceab7006000b800604288007a
:1048e400714288000700370011c0b30010c0b30044
:1048f40016fd070010c0b30050e8b70000c0eb007d
:10490400cceab7000080fa00000006000000fa00bc
:10491400f0558000000001000004e0000b003a00a4
:104924007fcabf008080fb00100020000100dd0072
:104934000080ea00800078007055800000806000ec
:10494400705588007cff0700240037007fcabf0031
:104954008080fb00100020000100dd008000780052
:1049640070558000008060000000e0001a003a00ea
:10497400c0558000000001000004e0001400320073
:104984007fcabf008080fb00100020000100dd0012
:104994008000780070558000008070007055880099
:1049a400950aa900952aa800954aa800956aa90025
:1049b40080c2b3009feab7000040eb00a0eab70052
:1049c40010c0b30050e8b7005dfe070003003700d5
:1049d40059ff07000100370059fe0700cccabf0089
:1049e4000080fb000080fa00000006000200fa00cc
:1049f40068cabf000080fb00000f78001e0078002a
:104a0400e20f50002f0032001e007800e20f500029
:104a140007003c001e0078000000e0000b0032009c
:104a24001e007800e10f50001b00320085003700a3
:104a34001e007800e30f50004a0032001e00780088
:104a4400e40f5000510032007e00370083cabf00db
:104a54006feab70084cabf006eeab70085cabf0018
:104a64006deab70086cabf006ceab70088cabf0007
:104a74006beab70089cabf006aeab7000040eb00de
:104a840050e8b7006000b8006042880071428800b6
:104a940010c0b30068eab700505380000000e00083
:104aa40003003a000040eb0068eab70065003700f5
:104ab400505380000000e9005053880020c0b30028
:104ac40068eab700505580000000e000060032009c
:104ad400505580009040900000c8b30000c06000b2
:104ae4000004e00057003a000356800022852000ad
:104af400605380007153800003000100e14f5000b7
:104b04000800320010c0b30050e8b7006000b800dd
:104b1400604288007142880010c0b30070eab70098
:104b240048003700605380007153800061004000ea
:104b3400e080480060538800715388000040eb0017
:104b440050e8b700002020000100200060428800e7
:104b540071428800208520003055880030c0b300a1
:104b640068eab7006042800071428000e00f5000a4
:104b7400e08f580003003a0010c0b30068eab700a1
:104b84003000370040c0b30068eab70050c8bf0027
:104b94000004e0002b003a0062428000734280006f
:104ba400f003200001002000800f5100818f590084
:104bb40024003600505580000000e000060032005a
:104bc400505580009040900000c8b30000c06000c1
:104bd4000004e0001b003a003255800003c4b30017
:104be40011c0b30010c0b3007ffc0700505588000b
:104bf40030c0b30068eab700d2538000e3538000aa
:104c040000fc2f00f1ff2f000200400083804800c9
:104c1400d0538800e15388006242800073428000d0
:104c240000fc2f00f1ff2f000200400083804800a9
:104c34006042880071428800305580000004b00052
:104c44003055880068cabf000080fb000080fa006d
:104c5400000006000200fa0069cabf000080fb00e1
:104c6400000f78001e007800e20f50007b00320035
:104c74001e007800e20f500007003c001e00780080
:104c84000000e0000b0032001e007800e10f50002d
:104c940018003200840037001e007800e30f500033
:104ca400220032001e007800e40f50004800320059
:104cb4007d00370083cabf006feab70084cabf0013
:104cc4006eeab70085cabf006deab70086cabf00a6
:104cd4006ceab70088cabf006beab70089cabf0094
:104ce4006aeab7000040eb0050e8b70010c0b30018
:104cf40070eab700505380000000e00003003a005f
:104d04000040eb0069eab7006700370030c0b30029
:104d140069eab70020852000305588000020200073
:104d240001002000604288007142880060428000d7
:104d340071428000e00f5000e08f580012003200f2
:104d4400405580000000e00006003200405580001d
:104d54009040900000c8b30000c060000004e00070
:104d640051003a003255800003c4b3008040eb0088
:104d740010c0b3001cfc07004055880040c0b300bd
:104d840069eab700120037001056800000000100e5
:104d94000004e0000b003200950aa900952aa8003f
:104da400954aa900956aa90070c2b3009feab700aa
:104db4000040eb00a0eab70010c0b30050e8b70011
:104dc4003900370020c0b30069eab7003600370065
:104dd400405580000000e00006003200405580008d
:104de4009040900000c8b30000c060000004e000e0
:104df4002d003a00d2538000e353800040558000d8
:104e0400104078000080fb000100200000005100e9
:104e140081805900d0538800e153880062428000a9
:104e24007342800040558000104078000080fb00f1
:104e34000100200000005100818059006042880078
:104e440071428800305580000004b000305588005d
:104e540030c0b30069eab70013003700245680005d
:104e64002285200060538000715380008041eb0054
:104e740004000100e14f50000b003a006053800031
:104e84007153800061004000e08048006053880056
:104e940071538800505380000000e900505388008b
:104ea40010c0b30069eab70069cabf000080fb0004
:104eb4000080fa00000006000000fa0031a920007a
:104ec4009140780000c8b30000c0600001c7b3007f
:104ed4000140700093eab70093eaa9000040eb0098
:104ee40094eab700950aa900952aa900954aa90051
:104ef400956aa90095aaa90095caa90095eaa900ee
:104f04000040eb0096eab7000040eb0097eab700d8
:104f14000040eb0098eab7000040eb0099eab700c4
:104f2400a0c0b3009aeab7009bcabf00604060000b
:104f34009beab7009ccabf00604060009ceab700cf
:104f44009dcabf00604060009deab7009ecabf00d2
:104f5400604060009eeab7000040eb009feab700a3
:104f64000040eb00a0eab7000040eb00a1eab70064
:104f74000040eb00a2eab7000040eb00a3eab70050
:104f84000040eb00a4eab7000080fa00000006002d
:020000040000fa
:104f94000000fa00eac2bf000004a2000080fb0087
:104fa400610060000080fa00000006000000fa00c2
:104fb400002020000080fa00000006000000fa0033
:104fc40030568000415680000080fa000000060040
:104fd4000000fa00e802a800ca22a800c822a9001a
:104fe400e822a8000080fa00000006001200fa007f
:104ff40010c0b3002047980030002000000f780054
:10500400ca22a8000000eb0010128800000520004e
:10501400200798002e0090000000e00020003a00d5
:1050240010128000f10320000100700010128800ab
:105034001b0037002e009000e80f50000c003600d3
:105044001e0fe9002e009000630060000000e000e5
:10505400030032002e0090006400400020079800f6
:105064002e0090004200de00200798000c0037005c
:105074002e0090004200dd000080ea007c00600009
:105084009e007000101280008080700000022000da
:1050940000807000101288000000eb0020079800c8
:1050a4002e0090000000e000e2ff3a000041eb0017
:1050b40031c0b300000220008d02070010c0b3000d
:1050c4005f0207000000eb0020079800050037008e
:1050d40000c0eb00b70207002e0090000000e800bb
:1050e400200798002e009000e90f5000f8ff3600ca
:1050f400ca22a90010c0b30051020700680047008b
:105104006011b8008040eb00600007004e00900082
:10511400300798006e409000e14f400006003200d6
:105124006e4090008080fb00700f200000806000c3
:10513400e10f5000070032000040eb0020479800c8
:10514400ca22a8002e4090000080fb00000f9800a7
:1051540046003700f0ff2000200798006a0047004f
:105164006011b80011c0b300480007005e00900051
:10517400300798002e0090000000e90020079800f6
:105184006e4090000004e000030032002e00900006
:105194000000e000f1ff3a002e0090000000e00063
:1051a40004003a000040eb0020479800ca22a800ff
:1051b4002b00370020c0b300210207000041eb00a0
:1051c40031c0b300e003200049020700111280003f
:1051d400b003200000807000101288006c004700ab
:1051e4006011b80061c1b300280007006e00900090
:1051f400300798006e0047000220200003002000c2
:1052040061c0b300210007007e00900030079800c1
:10521400f00f200020079800030037002e009000b4
:105224000000e900200798002e0090000000e00034
:10523400050032000001eb006000b800a200070086
:10524400e14f5000f5ff3a002e0090000000e0000e
:1052540003003a000040eb0020479800ca22a8004f
:105264002e4090000080fb00000f98000e08900074
:105274000080fa00000006000000fa001502070092
:10528400ca22a8000080fa00000006001600fa00f6
:10529400200f9800614f9800020f9800130f980098
:1052a4008000200010079800ca22a9006e489000d0
:1052b4000080fb00625529006600b900020040002e
:1052c40090407800660047006140980066004700ff
:1052d4000e0990009e099000120098002300980087
:1052e4006e4890000080fb00625529006600b900fa
:1052f400020040009040900066004700014878009a
:10530400e6004700310090000060a000b000980063
:1053140066004700604090002602070066004700d0
:105324005040900023020700660047004040900070
:105334002002070066004700304090001d0207006d
:1053440066004700204090001a02070066004700ec
:1053540010407800170207006e4890000080fb00a0
:10536400625529006600b9000080e80060007900f9
:105374000000e000080032006e4890000080fb004e
:10538400625529006600b9000080e80060007900d9
:10539400e10f50000c003a00c30107004047980099
:1053a4001e0090000000e900100798004e40900095
:1053b400e14f400011003a001e0090000000e000a0
:1053c400f5ff3a000d0037006e4890000080fb00a6
:1053d400625529006600b9000080e8006000790089
:1053e400e20f500005003a00af010700ae010700cc
:1053f40050479800ac010700404798006e48900061
:105404000080fb00625529006600b9000080e800b6
:1054140060007900e10f500019003a000040eb00f1
:10542400404798000040eb00004f78000e00370022
:105434000080eb00100798009b010700404798008c
:105444001e0090000000e900100798004e409000f4
:105454000004e00003003a001e0090000000e00099
:10546400f5ff3a001e4fe80080c1eb009ecf11000b
:10547400030032004e4090000004e000ecff3200d4
:1054840000c0eb00cb0107006e4890000080fb00d9
:10549400625529006600b900640040000200400023
:1054a400104078000004e00001003a00ca22a8007d
:1054b400ae0090002e089000010878002e0890009d
:1054c4000080fa00000006002000fa00200f980077
:1054d400310f9800420f980010c0b300404f98005d
:1054e4002e089000be0890004909dd00c700de00c8
:1054f400810071004900dd004007980051079800c1
:105504007a0047004e019000de01900071c0b300a4
:105514005eff07005e089000100f98002e50900068
:105524000004e0000d0032007c0047004e019000b2
:10553400de01900071c0b30054ff07006e089000b4
:10554400100f98002e5090000004e0000300320079
:105554008001eb00730f9800c7003700f02f200084
:10556400000f980000042000700798000300370023
:105574007e0090000000e900700798007e00900013
:105584000000e000faff3a0047010700504f98007e
:105594000e0890000000e900000f980000042000ad
:1055a40070079800030037007e0090000000e900b7
:1055b400700798007e0090000000e000faff3a00b7
:1055c4005e489000e14f400003003a000e0890004e
:1055d4000000e000ecff3a000e0890000000e0003c
:1055e400030032005e489000e24f400003003200a6
:1055f4000040eb00404f9800990037002e089000bf
:10560400be089000e00f5000e08f580006003a00fa
:105614004e0890000000e00003003a006000b8006b
:1056240030568800415688000000eb00000f9800b7
:10563400830037004e0890000000e0000c003200a8
:10564400f00f20004012880040c2bf00614060009b
:105654000004e000fcff32008e0890004e08900029
:10566400808040004012800080487800710037003c
:105674002e089000be089000e00f5000e08f580004
:105684006b003a008e089000601c2000808f500050
:105694000c0032008e089000601d2000808f5000a6
:1056a400080032008e089000601e2000808f500099
:1056b400040032008e089000601f2000808f50008c
:1056c40059003a00f80007000080fb0001002000a8
:1056d4002007980031079800f30007000080fb00c2
:1056e400010020004809dd00c801de0083017100cb
:1056f4004801dd002e009000be0090000200700002
:10570400838070002007980031079800e6000700a6
:105714000080fb0001002000c001dd000200200029
:105724002e009000be009000020070008380700084
:105734002007980031079800db0007000080fb0079
:1057440001002000c801dd00020020002e009000ae
:10575400be00900002007000838070002007980053
:1057640031079800d00007000080fb0001002000f2
:10577400008fbe00cc0007000080fb000100200069
:10578400c808dd000080fd00804078000040eb0088
:105794001e1f70001e977000c30007000080fb00ee
:1057a40001002000c000dd00000020001e1f70006a
:1057b4001e977000bc0007000080fb000100200061
:1057c400c800dd00000020001e1f70001e9770003e
:1057d4000e08900068004000000f98002e00900012
:1057e400be0090003e014000ae814800305680006b
:1057f40041568000800f5100818f59000d00360002
:105804002e009000be0090003e014000ae81480092
:105814000200be0061005000e0805800305688004d
:1058240041568800030037009f000700010037003d
:105834009d0007000e0890000000e800000f98008b
:105844008e089000f01f2000808f500079ff3600f2
:1058540000c0eb00d700070000c0eb00d500070034
:1058640000c0eb00d3000700ca22a8004e489000f5
:105874000080fb00700f98007e0890000080fa0002
:10588400000006001000fa00300798004107980055
:1058940052079800434f980010c0b300004f78009f
:1058a4003e009000ce009000e00f5000e08f5800c2
:1058b40006003a004e4890000004e00003003a005d
:1058c4000040eb00004f7800520037003e0090008b
:1058d400ce0090004909dd00c701de00830171009c
:1058e4004901dd006e00470091c0b30067fe070068
:1058f4007e009000200798004e4090000004e000d5
:10590400030032000040eb00004f780040003700f5
:10591400e0cfb300a70007000000eb0010079800d9
:105924000f0037009e0090005e0090000080400051
:10593400104078000080fb004012880040c2bf0085
:10594400614060000004e000fcff3200401280006f
:10595400104798001e0090000000e800100798000f
:105964009e009000f01f2000808f5000edff360055
:1059740000c0eb008f00070000c0eb008d000700a3
:1059840049000700104798001e4090000080fb006b
:105994006f006000e50f5000030032000040eb0090
:1059a400004f7800180037000000eb001007980043
:1059b400f00f20004012880040c2bf006140600028
:1059c4000004e000fcff3200401280001047980001
:1059d4001e0090000000e800100798001e40900090
:1059e4000004e00003003a001e0090000000e00004
:1059f400efff3a001e0090000000e00002003a00b1
:105a04000040eb00004f780000c0eb006900070085
:105a1400ca22a8001e80fb000080fa0000000600d5
:105a24000000fa00eac2bf000080fb000000d100c1
:105a3400614060000080fb000080fa000000060066
:105a44000800fa00604798006e40900040479800b4
:105a54000c003700b07c200001002000008fbe0045
:105a64000080eb008080eb001e0f40005e97480032
:105a74000080eb008080eb00be0f1000ae8f18009a
:105a8400f7ff3a004e4090000040e900404798007c
:105a94004e409000e14f4000eeff3a00000000004d
:105aa4000080fa00000006000000fa00f00f200059
:105ab4004012880040c2bf00614060000004e00062
:105ac400fcff3200401280000080fb000080fa00de
:105ad400000006000000fa0000128000f1ff270019
:105ae40001006000001288000080fa000000060037
:105af4000800fa00000f7800214798003247980008
:105b04000000eb00001288003e4090008080fb0003
:105b14001012800000807000101288002e40900047
:105b24000080fb00200798002e009000e20f500038
:105b3400090032002e009000e30f500008003200ec
:105b44002e0090000000e000010032000600370043
:105b54004302a8000400370042c2a8000200370034
:105b640042c2a8004302a9001e0078003007980032
:105b74003e009000e40f5000040032003e0090000c
:105b8400e50f50000200320004003700c822a800cc
:105b9400c802a8004322a90001003700c802a900d6
:105ba400e902a900d842a80041e2a8000080fa0056
:105bb400000006000400fa00204798002e409000e0
:105bc4000080fb004012880040c2bf0061406000ba
:105bd4000004e000fcff320040128000004f780017
:0c5be4000000eb000080fa00000006004a
:020000040000fa
:105bf0000000fa000300070039f407001b0007004b
:105c0000fdff37000000fa000080eb0060198800fb
:105c1000fdf30700816a20009140780000ccb300ba
:105c200000c060007041b300a8e6b700f16c20002e
:105c30009140780000ccb30000c060007040b30019
:105c4000cfe6b700016c20009140780000ccb30093
:105c500000c060000034a000c0e6b7007480a80057
:105c6000dcfc07000080fa00000006000000fa00db
:105c700010c8bf00ff4f50000600360088c4bf00a8
:105c8000624060000004e0000100320001003700c3
:105c9000fef807000080fa00000006000000fa008d
:105ca0000080fa00000006000000fa000080fa0000
:105cb000000006000000fa000080fa000000060064
:105cc0000000fa000080fa00000006000000fa0060
:105cd000d3f807000080fa00000006000000fa0078
:105ce0000080fa00000006000000fa00d1c1b300f5
:105cf00010c0b300f4f707009af807000080fa001c
:105d0000000006000000fa009444a8008070200003
:105d100050568800505680000000e9005056880018
:105d2000505680000000e000faff3a009444a900b9
:085d30000080fa0000000600eb
:020000040000fa
:105d3800b80a00000e00000002000000f827e0008a
:105d480027d82700ca2766002a122d00442c0000f5
:105d5800ca0a00000200000000000000000c000059
:105d680010000000000000000008000068020000a9
:105d780000000000cc0a0000020000000200000041
:105d8800ff000000680a000050000000000000004a
:105d9800c60a000004000000000000000000000027
:020000040000fa
:045da8000000fe00f9
:00000001FF
